:020000040800F2
:10000000680A0020890100086D05000869050008DC
:100010006B050008C3020008630D00080000000023
:10002000000000000000000000000000090C0008B3
:10003000C502000800000000EB0B0008C10C00081E
:10004000A3010008A3010008A3010008A301000800
:10005000A3010008A3010008A3010008A3010008F0
:10006000A3010008A3010008C9020008A3010008B9
:10007000A3010008A3010008A3010008A3010008D0
:10008000A3010008A3010008A3010008A3010008C0
:10009000A3010008A3010008A30100080903000848
:1000A000A3010008A3010008A3010008A3010008A0
:1000B000A3010008A3010008150D0008A301000812
:1000C000A3010008A3010008A3010008A301000880
:1000D000A3010008A3010008A3010008A301000870
:1000E000A3010008A3010008A301000800F002F822
:1000F00000F03AF80AA090E8000C82448344AAF188
:100100000107DA4501D100F02FF8AFF2090EBAE885
:100110000F0013F0010F18BFFB1A43F0010318473B
:10012000DC150000FC150000103A24BF78C878C127
:10013000FAD8520724BF30C830C144BF04680C60ED
:10014000704700000023002400250026103A28BF35
:1001500078C1FBD8520728BF30C148BF0B60704739
:100160001FB51FBD10B510BD00F076F81146FFF7A2
:10017000F7FF00F0F7FD00F094F803B4FFF7F2FF8B
:1001800003BC00F097F80000094880470948004781
:10019000FEE7FEE7FEE7FEE7FEE7FEE7FEE7FEE737
:1001A000FEE7FEE704480549054A064B7047000094
:1001B000C50C0008ED00000868040020680A002053
:1001C00068060020680600204FF0013C50F8042B20
:1001D00051F8043B9A4221D1A2EB0C03934313EA5A
:1001E000CC1317D150F8042B51F8043B9A4215D187
:1001F000A2EB0C03934313EACC130BD150F8042B5E
:1002000051F8043B9A4209D1A2EB0C03934313EA41
:10021000CC13DBD04FF00000704700BFD01A01BAFA
:10022000B1FA81F101F0180122FA01F0CB40C1F1DD
:100230002001DBB2C0B2C01A2CFA01F3D11A9143EB
:1002400011EAC311E6D1704770477047704700004C
:1002500000487047080400207546FFF7F9FFAE46D6
:1002600005006946534620F00700854618B020B5C2
:10027000FFF798FFBDE820404FF000064FF0000761
:100280004FF000084FF0000B21F00701AC46ACE83E
:10029000C009ACE8C009ACE8C009ACE8C0098D46AB
:1002A000704710B50446AFF300802046BDE810400B
:1002B000FFF763BF01491820ABBEFEE7260002002E
:1002C0007047FEE77047000010B5102000F042F8BC
:1002D000012813D10A4C1021204600F038F940B90A
:1002E0002021204600F033F918B906480188491E3C
:1002F0000180BDE81040102000F026B810BD0000BD
:10030000000801400400002010B5202000F022F871
:10031000012813D10A4C2021204600F018F940B9D9
:100320001021204600F013F918B906480188491C2D
:100330000180BDE81040202000F006B810BD00008C
:1003400000080140040000200149086070470000D7
:100350001404014001460020054A12680A40044B7B
:1003600014331B680B4202D0002A00D001207047D2
:100370000004014030B51B4A83790168002B2AD064
:1003800013688B431360111D0B680468A3430B6053
:10039000017911440B68046823430B60114C083445
:1003A0002168036899432160231D19680568A943E2
:1003B00019604179102905D011440A680068024388
:1003C0000A6030BD21680268114321601968006825
:1003D0000143196030BD0079104402688A4302600D
:1003E00030BD0000000401401FB50121042000F0D1
:1003F000FDFB0121084600F0F9FB48208DF80F00B5
:100400003024ADF80C4003208DF80E0003A91B48E2
:1004100000F04AF80421002000F032F80521002005
:1004200000F02EF8019401248DF80A4000208DF888
:1004300008000C208DF8090001A8FFF79BFF4FF47E
:10044000A06000F0C7F80A208DF800008DF8034086
:100450008DF801408DF80240684600F089F81720B9
:100460008DF800008DF803408DF8014002208DF8D2
:100470000200684600F07CF81FBD00000008014043
:1004800010B58A07120F0F23934021F0030405498A
:1004900021448C689C438C608B68904003438B6044
:1004A00010BD0000000001402DE9F0410022CC7891
:1004B00004F00F03E40601D58C7823430C784FF049
:1004C0000F0714F0FF0F4FF0010C1CD005680CFA59
:1004D00002F40E882640A64211D1960007FA06F8CB
:1004E00025EA080503FA06F848EA0505CE78282E1D
:1004F00002D0482E02D002E0446100E00461521CA8
:10050000082AE4D305600A88FF2A1ED9456800221C
:1005100002F108060CFA06F40E882640A64210D115
:10052000960007FA06F825EA080503FA06F848EAED
:100530000505CE78282E00D14461CE78482E00D112
:100540000461521C082AE3D34560BDE8F0810246ED
:10055000002092680A4200D001207047002A01D092
:100560000161704741617047FEE7FEE77047000098
:1005700070B50F23C27801260178002A1ED0144AD4
:10058000126802F4E062C2F5E062120AC2F10404E9
:10059000D3404578A54082781A402A43120101F1E0
:1005A000E02181F80024007800F01F018E4040090E
:1005B000800000F1E020C0F8006170BD01F01F0074
:1005C00086404809800000F1E020C0F8806170BDDD
:1005D0000CED00E002490843024908607047000042
:1005E0000000FA050CED00E010B50021074C0022D8
:1005F000002004EBC1131A54401CC0B28028FAD367
:10060000491CC9B20829F3D310BD0000080000201E
:100610002DE9F0417F2828D83F2926D88418802C3E
:1006200002D9C0F18002D2B2CC18402C02D9C1F15B
:100630004003DBB201250E4E871801EB030812E0E0
:10064000044601F0070205FA02FCCA0806EBC212D2
:1006500005E0135D23EA0C031355641CE4B2A742C2
:10066000F7D8491CC9B28845EAD8BDE8F081000036
:100670000800002038B500214FF47A720020401C99
:100680009042FCD3491C9142F8D30121082000F08C
:10069000ADFA14208DF8030003208DF8020002202B
:1006A000ADF80000094C69462046FFF7FDFE211514
:1006B000ADF8001069462046FFF7F6FE012000F075
:1006C0005BFA012000F060FA38BD0000000C014028
:1006D00070B505460024802626FA04F0284000D094
:1006E000012000F051FA012000F046FA002000F04D
:1006F00043FA641CE4B2082CEED3012000F03CFA6B
:10070000BDE87040002000F037BA10B5012000F0BD
:100710003BFA012000F030FA002000F035FABDE885
:100720001040002000F028BA10B5002000F02CFA8C
:10073000012000F021FABDE81040012000F024BAA9
:1007400010B5FFF797FFAE2000F026FAD52000F095
:1007500023FA802000F020FAA82000F01DFA3F20A4
:1007600000F01AFAD32000F017FA002000F014FA73
:10077000402000F011FAA12000F00EFAC82000F08D
:100780000BFADA2000F008FA122000F005FA8120B6
:1007900000F002FACF2000F0FFF9D92000F0FCF9B8
:1007A000F12000F0F9F9DB2000F0F6F9302000F03C
:1007B000F3F9A42000F0F0F9A62000F0EDF98D2067
:1007C00000F0EAF9142000F0E7F9AF2000F0E4F9B6
:1007D000FFF70AFFBDE8104000F0BAB92DE9F84371
:1007E0000746884691460024104E06E028464946B2
:1007F000FFF7EAFC60B1641CE4B204EBC40006EB52
:100800008000203005460AA1FFF7DEFC0028EDD16C
:1008100004EBC40006EB80000090102308F0FF01F9
:10082000F8B21A4600F07CF8BDE8F883B00D000875
:100830000000000010B50C4640F0B00000F0ACF92C
:10084000102040EA141000F0A7F904F00F00BDE8F2
:10085000104000F0A1B9000008B5203A082B0CD0D8
:10086000062B09D1094B02EB420203EB4202009234
:100870000823062200F054F808BD054B03EB0212D2
:1008800000921023082200F04BF808BDC0140008A5
:10089000D00E00082DE9FC5F81468B46924600256C
:1008A000002001900026DFF870802EE001A9485555
:1008B0006D1CEDB2032D26D30025002406E038463A
:1008C00001A9FFF781FC60B1641CE4B204EBC40031
:1008D00008EB8007203711A13846FFF775FC002888
:1008E000EDD1701C0321B0FBF1F004EBC401401EFC
:1008F00008EB810109EB001010230091C0B21A46E9
:10090000594600F00DF8761CF6B21AF806000028D9
:10091000CCD1BDE8FC9F0000B00D00080000000035
:100920002DE9FF4F83B0154698464CB203987F28B7
:100930007DD8002600274FF00109002C18DACDF8E9
:10094000048008EB040000F0FF08641C6042C1173B
:1009500000EB517109EBE102D6B221F00701401A18
:10096000401CC7B200244FFA88F001285FDB01E089
:100970003F2C5CDCE1B243462A460398FFF748FE71
:10098000A8F101084FEAE87008EB507009EBE000AD
:10099000C0B20090002171E000236BE0039818447E
:1009A0007F2869D8E21704EB527201EBE208B8F134
:1009B000070F66DC3EB301EBE20C334ADDF84090F2
:1009C00002EBCC1C8A19A2F1010A0AFB05FA994430
:1009D0001CF800801AF809A02AFA07FA48EA0A085F
:1009E0000CF80080DDF804A0BAEBC20F40D96A43CE
:1009F00012F80920C7F1080902FA09F248EA0208C8
:100A00000CF8008034E0DDF8409001FB05FC9944CF
:100A100022F0070A1CF809B0DFF86CE0A4EB0A0A20
:100A200001EBE2020BFA0AFB0EEBC21E00E028E02B
:100A3000CDF808E01EF800E04BEA0E0BDDF808E008
:100A40000EF800B008F10108B8F1070F10DC1CF82F
:100A500009C0CAF108082CFA08FCDFF82C80521CE7
:100A600008EBC21212F800804CEA080C02F800C031
:100A70005B1CDBB2AB4291D3491CC9B200988142E6
:100A80008AD307B0BDE8F08F080000202DE9F843B5
:100A900081460F4690461E460025002452E00A2853
:100AA00007D1082E37D008203844C7B200246D1C67
:100AB000EDB2601C00FB0690802805D9082E2CD0D2
:100AC00008203844C7B2002479B240293EDC18F827
:100AD00005207E2A2BD90020009018F805008DF8FB
:100AE00000006D1CE8B218F800208DF80120401CB1
:100AF000C5B218F805008DF80200082E0FD004FBCF
:100B0000069040B233466A46FFF768FE6D1CEDB2B0
:100B1000A41CE4B216E01020C6E71020D1E704FBC5
:100B2000069040B233466A46FFF758FEEEE704FBF4
:100B30000690C0B233463946FFF78EFE6D1CEDB20B
:100B4000641CE4B218F805000028A8D1BDE8F883B9
:100B500070B50024074D00212046FFF76BFE05EB22
:100B6000C410802100F029F8641CE4B2082CF2D3F0
:100B700070BD000008000020024602210148FFF776
:100B8000EDBC0000000C014002464FF480610148BA
:100B9000FFF7E4BC000C014010B50446FFF7B5FDBB
:100BA0007820FFF795FD0020FFF792FD2046FFF724
:100BB0008FFDBDE81040FFF7B7BD70B505460E4686
:100BC000FFF7A3FD7820FFF783FD4020FFF780FDAE
:100BD000002404E0285DFFF77BFD641CE4B2B4420E
:100BE000F8D3BDE87040FFF79FBD7047054A002964
:100BF00003D091690143916170479169814391618B
:100C00007047000000100240704700F001B800007B
:100C10000CB50022019200922748016841F480310E
:100C200001604FF4A063016801F400310091019963
:100C3000491C0191009911B901999942F3D10168B8
:100C4000890302D50121009100E000920099012959
:100C500030D11A490A6842F010020A600A6822F08C
:100C600003020A600A6842F002020A6041684160B9
:100C700041684160416841F480614160416821F40C
:100C80007C114160416841F4E8114160016841F024
:100C90008071016001688901FCD5416821F0030180
:100CA0004160416841F0020141604168C1F3810146
:100CB0000229FAD10CBD00000010024000200240C1
:100CC0007047000010B50F48016841F00101016054
:100CD00041680D4A1140416001680C4A11400160B1
:100CE000016821F480210160416821F4FE01416026
:100CF0004FF41F018160FFF788FF05494FF0006046
:100D0000086010BD001002400000FFF8FFFFF6FE73
:100D100008ED00E010B5094C0121204600F015F85F
:100D200001280AD1064841880180002141802046DF
:100D3000BDE81040012100F005B810BD00080040DA
:100D400000000020C9430182704702460020138A38
:100D50000B4092890A40002B02D0002A00D00120CB
:100D60007047FEE7FFF7ECFCFFF73EFB09A21921F5
:100D70000020FFF78FFD082308A219212320FFF789
:100D800085FE08A219215020FFF784FDFFF7E0FE41
:100D9000FCE70000E5AE9EE78EB00000332E38562B
:100DA00000000000E794B5E58E8BE580BC000000F4
:100DB000100C048414640506F404040404140C00E8
:100DC000048484444724140C070C14244484040031
:100DD000E5AE9E00048484FC848400FE0202F202DC
:100DE00002FE00002060201F109040231806017EA4
:100DF0008083E000E78EB0008080808080808080EB
:100E00008080808080808000000000000000000062
:100E10000000000000000000E4B880008080402056
:100E2000100804C304081020408080000000000067
:100E3000000000FF0000000000000000E4B8AA006D
:100E40000000F888888888FF88888888F800000073
:100E500000001F080808087F888888889F80F000A5
:100E6000E794B5000000FE0282828282FA828282CA
:100E70008282020080601F40404040407F404044EA
:100E800058404000E58E8B00008060F80704E4A421
:100E9000A4BFA4A4E4040000010000FF40407F4A76
:100EA0004A4A4A4A7F404000E580BC00FF010101F8
:100EB0003109090909897101010101FFFF80808061
:100EC0008080809681808080808080FF000000008C
:100ED0000000000000000000000000000000000012
:100EE000000000F8000000000000003330000000A7
:100EF00000160E00160E00000000000000000000AA
:100F000040C07840C0784000043F04043F0404001F
:100F1000007088FC08300000001820FF211E00002F
:100F2000F008F000E018000000211C031E211E0044
:100F300000F00888700000001E21232419272110CA
:100F4000000000160E00000000000000000000007D
:100F5000000000E018040200000000071820400014
:100F600000020418E0000000004020180700000004
:100F7000404080F0804040000202010F0102020068
:100F8000000000F0000000000101011F010101004C
:100F9000000000000000000000B070000000000031
:100FA000000000000000000000010101010101013A
:100FB00000000000000000000030300000000000D1
:100FC00000000000806018040060180601000000A6
:100FD00000E010080810E000000F102020100F00A3
:100FE000001010F8000000000020203F202000002A
:100FF0000070080808887000003028242221300082
:1010000000300888884830000018202020110E0089
:101010000000C02010F8000000070424243F240032
:1010200000F80888880808000019212020110E0007
:1010300000E0108888180000000F112020110E0019
:1010400000380808C83808000000003F0000000011
:101050000070880808887000001C222121221C00D2
:1010600000E010080810E0000000312222110F00FB
:10107000000000C0C0000000000000303000000090
:10108000000000C0C0000000000080B07000000040
:101090000000804020100800000102040810200019
:1010A0004040404040404000040404040404040064
:1010B00000081020408000000020100804020100F9
:1010C000007048080808F0000000003036010000F9
:1010D000C030C828E810E0000718272423140B00AC
:1010E0000000C038E0000000203C23020227382026
:1010F00008F8888888700000203F202020110E000A
:10110000C030080808083800071820202010080000
:1011100008F808080810E000203F202020100F00E9
:1011200008F88888E8081000203F202023201800B5
:1011300008F88888E8081000203F2000030000001D
:10114000C03008080838000007182020221E0200BE
:1011500008F808000008F808203F210101213F207D
:10116000000808F8080800000020203F20200000A8
:1011700000000808F8080800C08080807F00000098
:1011800008F888C028180800203F200126382000D1
:1011900008F8080000000000203F20202020300038
:1011A00008F8F800F8F80800203F003F003F200052
:1011B00008F830C00008F808203F200007183F005A
:1011C000E01008080810E0000F10202020100F0089
:1011D00008F808080808F000203F2101010100007C
:1011E000E01008080810E0000F18242438504F00C1
:1011F00008F8888888887000203F2000030C302081
:1012000000708808080838000038202121221C00BE
:10121000180808F8080818000000203F2000000007
:1012200008F808000008F808001F202020201F00F0
:101230000878880000C83808000007380E01000050
:10124000F80800F80008F800033C0700073C03001A
:10125000081868808068180820302C03032C302080
:101260000838C800C83808000000203F20000000EF
:1012700010080808C8380800203826212020180047
:10128000000000FE020202000000007F404040001B
:10129000000C30C000000000000000010638C00053
:1012A00000020202FE000000004040407F000000FB
:1012B00000201008040810200000000000000000BA
:1012C000000000000000000080808080808080801E
:1012D0000002040800000000000000000000000000
:1012E00000008080808000000019242222223F20FC
:1012F00008F8008080000000003F112020110E003F
:101300000000008080800000000E112020201100CD
:10131000000000808088F800000E112020103F207F
:101320000000808080800000001F22222222130003
:10133000008080F0888888180020203F202000004E
:101340000000808080808000006B94949493600003
:1013500008F8008080800000203F210000203F200E
:1013600000809898000000000020203F202000000E
:10137000000000809898000000C08080807F0000FE
:1013800008F8000080808000203F24022D302000DB
:10139000000808F8000000000020203F2020000086
:1013A0008080808080808000203F20003F20003FA0
:1013B000008080008080000000203F2100203F202E
:1013C0000000808080800000001F202020201F005F
:1013D000808000808000000080FFA12020110E008E
:1013E0000000008080808000000E112020A0FF807F
:1013F000808080008080800020203F21200001002C
:101400000000808080808000003324242424190080
:10141000008080E0808000000000001F202000008D
:101420008080000000808000001F202020103F20CE
:10143000808080000080808000010E30080601005E
:1014400080800080008080800F300C030C300F0003
:1014500000808000808080000020312E0E3120002E
:10146000808080000080808080818E70180601005E
:1014700000808080808080000021302C222130007C
:1014800000000000807C020200000000003F40409D
:1014900000000000FF00000000000000FF0000004E
:1014A0000002027C800000000040403F000000007D
:1014B000008040408000008000000000000101002A
:1014C0000000000000000000002F000000000700E6
:1014D000070000147F147F1400242A7F2A1200239F
:1014E00013086462003649552250000000070000CE
:1014F00000001C224100000041221C000014083E94
:1015000008140008083E0808000000A06000000859
:1015100008080808000060600000002010080402AD
:10152000003E5149453E0000427F4000004261516B
:101530004946002141454B31001814127F10002705
:1015400045454539003C4A494930000171090503C8
:1015500000364949493600064949291E00003636F9
:10156000000000005636000000081422410000145C
:101570001414141400004122140800020151090639
:10158000003E4955592E007C1211127C007F4949BA
:101590004936003E41414122007F4141221C007FEB
:1015A00049494941007F09090901003E4149497AF9
:1015B000007F0808087F0000417F41000020404173
:1015C0003F01007F08142241007F40404040007FDF
:1015D000020C027F007F0408107F003E4141413E23
:1015E000007F09090906003E4151215E007F09196B
:1015F00029460046494949310001017F0101003F68
:101600004040403F001F2040201F003F4038403FE7
:10161000006314081463000708700807006151494B
:10162000454300007F4141000002040810200000F3
:1016300041417F000004020102040040404040405C
:10164000000001020400002054545478007F4844F4
:10165000443800384444442000384444487F00382B
:101660005454541800087E0901020018A4A4A47C54
:10167000007F080404780000447D4000004080841E
:101680007D00007F102844000000417F4000007C66
:1016900004180478007C0804047800384444443872
:1016A00000FC242424180018242418FC007C0804BE
:1016B000040800485454542000043F444020003C97
:1016C0004040207C001C2040201C003C4030403C1E
:1016D000004428102844001CA0A0A07C00446454AE
:1016E0004C440000087F41000000007F0000000023
:1016F000417F080000080408100800001C170008BB
:10170000000000200800000028010008241700083D
:1017100008000020600A00004401000800000000EA
:0417200000000000C5
:04000005080000ED02
:00000001FF
